:020000040000FA
:0200000038289E
:040002000034003492
:080008008B13A200030EA300FC
:100010000C1C112821088F0020088E002030850636
:100020000C10230E8300A20E220E8B1709008312E0
:10003000850107309900831600009F011F3085005D
:10004000FF2390000C1481131514951415159515A4
:10005000151683120B178B17013090000800E23041
:10006000A400D930A500F030A6001F30A70008007A
:100070002F20051C42282408A1008F002508A0007D
:100080008E0048282608A1008F002708A0008E00B7
:100090001720051C50282408A1002508A000492885
:0A00A0002608A1002708A000492847
:02400E00943FDD
:00000001FF
